:1000000012C0C9C02BC02AC029C028C027C026C022
:10001000A8C02EC123C022C021C020C01FC01EC046
:100020001DC01CC01BC011241FBECFE5D4E0DEBF25
:10003000CDBF10E0A0E6B0E0E6EEF1E102C0059031
:100040000D92AA36B107D9F710E0AAE6B0E001C0D8
:100050001D92A237B107E1F71BD1C3C8D1CFDF93FF
:10006000CF93CDB7DEB787E390E02FEFFC0120837D
:1000700088E390E0FC01108284E390E02FEFFC0124
:10008000208385E390E0FC01108281E390E020E38F
:10009000FC01208382E390E0FC011082CF91DF918C
:1000A0000895DF93CF93CDB7DEB782E390E022E3EC
:1000B00030E0F90120812061FC012083CF91DF91A4
:1000C0000895DF93CF93CDB7DEB782E390E022E3CC
:1000D00030E0F90120812F7EFC012083CF91DF9158
:1000E0000895DF93CF93CDB7DEB785E390E025E3A6
:1000F00030E0F90120812062FC012083CF91DF9163
:100100000895DF93CF93CDB7DEB785E390E025E385
:1001100030E0F90120812F7DFC012083CF91DF9118
:100120000895DF93CF93CDB7DEB785E390E025E365
:1001300030E0F90120812860FC012083CF91DF911C
:100140000895DF93CF93CDB7DEB785E390E025E345
:1001500030E0F9012081277FFC012083CF91DF91DE
:1001600008951F920F920FB60F9211248F939F93B1
:10017000DF93CF93CDB7DEB780EA9FE090936C001A
:1001800080936B00CF91DF919F918F910F900FBE65
:100190000F901F9018951F920F920FB60F92112477
:1001A0002F938F939F93EF93FF93DF93CF9300D081
:1001B000CDB7DEB780E390E0FC018081882F90E02E
:1001C00084709070009759F08CE490E0FC011182EB
:1001D00010828EE490E021E0FC0120833BC080E3AC
:1001E00090E0FC018081882F90E0847090700097EF
:1001F00089F58EE490E0FC0110828CE490E0FC0133
:10020000808191819A83898389819A81FDE78130F8
:100210009F0738F088EE93E090936C0080936B001A
:1002200019C089819A812EE38038920728F41092B0
:100230006C0010926B000EC089819A8180589E4399
:10024000929582958F7089279F70892790936C0073
:1002500080936B000F900F90CF91DF91FF91EF9102
:100260009F918F912F910F900FBE0F901F90189517
:100270001F920F920FB60F921124DF93CF93CDB739
:10028000DEB7CF91DF910F900FBE0F901F901895A2
:100290000F931F93DF93CF93CDB7DEB7E8970FB6D9
:1002A000F894DEBF0FBECDBFDADE85E590E021E039
:1002B000FC0120838BE590E020E4FC0120838FE4A7
:1002C00090E0FC01108289E590E029E530E0F90139
:1002D00020812460FC0120838EE490E0FC011082E8
:1002E0008CE490E0FC011182108283E590E021E033
:1002F000FC01208389E590E029E530E0F9012081C7
:100300002160FC01208378948EE490E021E0FC01E0
:100310002083D7DEF6DE15DF01C0000080916B0080
:1003200090916C00F3E085389F0710F0FADE01C071
:1003300008DF80916B0090916C0022E08D3B92076A
:1003400010F0CFDE01C0DDDE80916B0090916C007B
:10035000893C910508F4ECC180E090E0AAEFB3E499
:1003600089839A83AB83BC8369817A818B819C81E9
:1003700020E030E04AE755E4A9D3DC01CB018D83CE
:100380009E83AF83B88711E06D817E818F819885D0
:1003900020E030E040E85FE3E4D488230CF010E094
:1003A000112329F081E090E09A87898742C011E00B
:1003B0006D817E818F81988520E03FEF4FE757E484
:1003C0007AD418160CF010E0112351F169817A816A
:1003D0008B819C8120E030E040E251E477D3DC0166
:1003E000CB01BC01CD01B0D1DC01CB019A8789875B
:1003F00012C080E991E09C878B878B859C858C015E
:10040000C8010197F1F78C011C870B8789859A85B4
:1004100001979A87898789859A85009751F716C031
:100420006D817E818F8198858FD1DC01CB019A8788
:10043000898789859A859E878D878D859E858C0184
:10044000F8013197F1F78F011E870D872ADE80E0D2
:1004500090E0A0EAB1E48F87988BA98BBA8B6F8567
:10046000788989899A8920E030E04AE755E42ED3DB
:10047000DC01CB018B8B9C8BAD8BBE8B11E06B8930
:100480007C898D899E8920E030E040E85FE369D473
:1004900088230CF010E0112329F081E090E0988F80
:1004A0008F8B42C011E06B897C898D899E8920E009
:1004B0003FEF4FE757E4FFD318160CF010E011237D
:1004C00051F16F85788989899A8920E030E040E28E
:1004D00051E4FCD2DC01CB01BC01CD0135D1DC0102
:1004E000CB01988F8F8B12C080E991E09A8F898F12
:1004F000898D9A8D8C01C8010197F1F78C011A8FB3
:10050000098F8F89988D0197988F8F8B8F89988D00
:10051000009751F716C06B897C898D899E8914D10B
:10052000DC01CB01988F8F8B8F89988D9C8F8B8F5F
:100530008B8D9C8D8C01F8013197F1F78F011C8F09
:100540000B8FBFDD80E090E0A4E3B3E48D8F9E8F3E
:10055000AF8FB8A36D8D7E8D8F8D98A120E030E098
:100560004AE755E4B3D2DC01CB0189A39AA3ABA33C
:10057000BCA311E069A17AA18BA19CA120E030E08D
:1005800040E85FE3EED388230CF010E0112329F05C
:1005900081E090E09EA38DA342C011E069A17AA101
:1005A0008BA19CA120E03FEF4FE757E484D31816BE
:1005B0000CF010E0112351F16D8D7E8D8F8D98A17F
:1005C00020E030E040E251E481D2DC01CB01BC010B
:1005D000CD01BAD0DC01CB019EA38DA312C080E96E
:1005E00091E098A78FA38FA198A58C01C8010197CE
:1005F000F1F78C0118A70FA38DA19EA101979EA3CF
:100600008DA38DA19EA1009751F716C069A17AA173
:100610008BA19CA199D0DC01CB019EA38DA38DA1C0
:100620009EA19AA789A789A59AA58C01F80131975F
:10063000F1F78F011AA709A734DD80E090E0A0EA66
:10064000B1E48BA79CA7ADA7BEA76BA57CA58DA584
:100650009EA520E030E04AE755E438D2DC01CB012A
:100660008FA798ABA9ABBAAB11E06FA578A989A900
:100670009AA920E030E040E85FE373D388230CF0D0
:1006800010E0112329F081E090E09CAB8BAB42C0DD
:1006900011E06FA578A989A99AA920E03FEF4FE75B
:1006A00057E409D318160CF010E0112351F16BA593
:1006B0007CA58DA59EA520E030E040E251E406D265
:1006C000DC01CB01BC01CD013FD0DC01CB019CABF7
:1006D0008BAB12C080E991E09EAB8DAB8DA99EA93A
:1006E0008C01C8010197F1F78C011EAB0DAB8BA9F2
:1006F0009CA901979CAB8BAB8BA99CA9009751F748
:1007000016C06FA578A989A99AA91ED0DC01CB01D2
:100710009CAB8BAB8BA99CA998AF8FAB8FA998ADE5
:100720008C01F8013197F1F78F0118AF0FABC9DCDD
:1007300080916B0090916C00893C910508F0EDCDA3
:10074000C0DCDFDCFEDCEACDEF92FF920F931F935B
:100750007B018C0120E030E040E05FE4D7D287FDF0
:100760000FC0C801B70120E030E040E05FE483D172
:1007700023D39B01AC01205030404040504805C07D
:10078000C801B70119D39B01AC01B901CA011F917E
:100790000F91FF90EF900895A0E0B0E0E1EDF3E05D
:1007A000EDC4FC01EA018081823008F438C1DB012C
:1007B0009C91923008F430C1843059F4943009F09F
:1007C0002EC1918111968C911197981709F021C132
:1007D00026C1943009F420C19230B1F4823009F07E
:1007E0001EC1CA01AF0128E0DA010D90AD01DC01A4
:1007F0000D92CD012150C1F7DB0111968C9111971B
:100800009181892389830AC1823009F405C1C2809C
:10081000D380DB0112966D907C90139724813581F3
:10082000468157811496ED90FD900D911C9117977C
:10083000C601861997095C0197FF04C0AA24BB244E
:10084000A81AB90AB0E2AB16B1040CF061C01816D0
:1008500019066CF5370148010A2C04C09694879458
:10086000779467940A94D2F781E090E0A0E0B0E03A
:100870000A2C04C0880F991FAA1FBB1F0A94D2F725
:100880000197A109B1098E219F21A023B123EE2454
:10089000FF248701E3940097A105B10519F4EE2424
:1008A000FF248701E628F728082919293CC000976A
:1008B000D1F1CA0CDB1C39014A010A2C04C0969400
:1008C0008794779467940A94D2F781E090E0A0E04F
:1008D000B0E00A2C04C0880F991FAA1FBB1F0A94FE
:1008E000D2F70197A109B10982239323A423B52349
:1008F00021E030E040E050E00097A105B10519F497
:1009000020E030E0A90126293729482959290BC0C0
:100910006C147D0424F4EE24FF24870104C06301D9
:1009200020E030E0A9018181FB019181891709F460
:1009300045C0882349F0D801C701821B930BA40B43
:10094000B50B9C01AD0104C02E193F09400B510BA2
:1009500057FD04C01982DB82CA820BC081E0898303
:10096000DB82CA8250954095309521953F4F4F4F7D
:100970005F4F2C833D834E835F830DC0880F991F8B
:10098000AA1FBB1F8C839D83AE83BF838A819B81FB
:1009900001979B838A838C819D81AE81BF819C015D
:1009A000AD0121503040404050402F3FEFEF3E0717
:1009B000EFEF4E07EFE35E0708F30BC08983DB829E
:1009C000CA822E0D3F1D401F511F2C833D834E8335
:1009D0005F8383E088832C813D814E815F8157FF57
:1009E0001DC0DA01C90181709070A070B070569579
:1009F000479537952795822B932BA42BB52B8C836A
:100A00009D83AE83BF838A819B8101969B838A836A
:100A100005C0E2E6F0E003C0FB0101C0FE01CF012A
:100A2000CDB7DEB7EEE0C6C3A0E2B0E0E9E1F5E0A5
:100A3000ADC369837A838B839C832D833E834F83ED
:100A4000588789E0E82EF12CEC0EFD1ECE010196B0
:100A5000B701CED28E010F5E1F4FCE010596B801B1
:100A6000C7D2C701B801AE01475E5F4F95DEF3D133
:100A7000A096E6E0A7C3A0E2B0E0E0E4F5E086C31C
:100A800069837A838B839C832D833E834F8358872E
:100A90008E01075F1F4FCE010196B801A9D291E1E7
:100AA000E92EF12CEC0EFD1ECE010596B701A0D269
:100AB0008A8991E089278A8BC801B701AE01475E18
:100AC0005F4F6ADEC8D1A096E6E07CC3A0E2B0E04A
:100AD000EBE6F5E04FC369837A838B839C832D8398
:100AE0003E834F835887CE010196BE01675F7F4FDB
:100AF0007FD2CE010596BE016F5E7F4F79D2998578
:100B0000923078F089898230C0F0943019F48230C4
:100B100041F4CBC0843019F4923079F4C6C09230DD
:100B200051F481E02A859A89291709F480E08A879F
:100B3000CE010996BCC0823051F481E02A859A89A1
:100B4000291709F480E08A8BCE014196B0C06D84EC
:100B50007E848F849888ED88FE880F89188DE0E266
:100B6000F0E080E090E0DC01AA24BB24650120E0F5
:100B700030E0A901B3016170707061157105D1F0A9
:100B80002E0D3F1D401F511F15012601280E391E35
:100B90004A1E5B1E81E090E0A0E0B0E02E153F050C
:100BA0004007510718F080E090E0DC01820D931DB2
:100BB000A41DB51DAA0CBB1CCC1CDD1C17FF09C055
:100BC00061E0262E312C412C512CA228B328C428B8
:100BD000D528319749F0EE0CFF1C001F111F969489
:100BE000879477946794C6CF6B897C89EB85FC8565
:100BF0006E0F7F1F6E5F7F4F7C8F6B8F61E0EA858A
:100C00007A89E71709F460E06A8F6B8D7C8D10C0DC
:100C1000FC01E170F070309729F0569547953795B3
:100C200027955068B695A795979587956F5F7F4FE5
:100C3000B7FDEECF0CC0880F991FAA1FBB1F57FD31
:100C40008160220F331F441F551F61507040803058
:100C5000E0E09E07E0E0AE07E0E4BE0760F36B8FE4
:100C60007C8F6FE7E62EF12C012D112DE822F92261
:100C70000A231B2360E4E616F1040105110561F463
:100C800087FD0AC0211531054105510529F0805C19
:100C90009F4FAF4FBF4F80788D8F9E8FAF8FB8A380
:100CA00083E0898FCE01499602C082E690E0D3D0DE
:100CB000A096E2E17BC2A8E1B0E0E0E6F6E066C221
:100CC00069837A838B839C832D833E834F835887EC
:100CD0008E01075F1F4FCE010196B80189D181E1D6
:100CE000E82EF12CEC0EFD1ECE010596B70180D149
:100CF0008985823038F08989823020F0C801B701B7
:100D0000E0D101C08FEF6896E6E05CC2A8E1B0E0F8
:100D1000EBE8F6E03BC269837A838B839C832D8367
:100D20003E834F8358878E01075F1F4FCE01019688
:100D3000B8015ED181E1E82EF12CEC0EFD1ECE0152
:100D40000596B70155D18985823038F0898982307E
:100D500020F0C801B701B5D101C08FEF6896E6E079
:100D600031C2A8E1B0E0E6EBF6E010C269837A8315
:100D70008B839C832D833E834F8358878E01075F2F
:100D80001F4FCE010196B80133D181E1E82EF12C3D
:100D9000EC0EFD1ECE010596B7012AD18985823061
:100DA00038F08989823020F0C801B7018AD101C0AA
:100DB00081E06896E6E006C2ACE0B0E0E1EEF6E085
:100DC000E9C169837A838B839C83CE010196BE013E
:100DD0006B5F7F4F0DD18D81823081F1823070F158
:100DE000843021F48E81882369F10AC02F813885EF
:100DF00037FD24C06E812F3131053CF0662311F19F
:100E000020E030E040E050E821C08EE190E0821B1D
:100E1000930B29853A854B855C8504C0569547958B
:100E2000379527958A95D2F7662381F0509540959E
:100E3000309521953F4F4F4F5F4F08C020E030E085
:100E4000A90104C02FEF3FEF4FEF5FE7B901CA01DF
:100E50002C96E2E0BBC1EF92FF920F931F93CF93CA
:100E6000DF93FC0124813581468157816181808136
:100E7000823020F44061EFEFF0E0A3C0843009F449
:100E80009BC0823009F492C02115310541055105FE
:100E900009F48FC00280F381E02D8FEFE238F8076C
:100EA0000CF05AC0C2E8DFEFCE1BDF0BCA31D10510
:100EB0006CF579018A010C2E04C016950795F794FC
:100EC000E7940A94D2F781E090E0A0E0B0E00C2E25
:100ED00004C0880F991FAA1FBB1F0A94D2F701975D
:100EE000A109B10982239323A423B52321E030E093
:100EF00040E050E00097A105B10519F420E030E092
:100F0000A9012E293F29402B512B03C020E030E0BE
:100F1000A901DA01C9018F779070A070B070803498
:100F20009105A105B10539F427FF09C0205C3F4FA9
:100F30004F4F5F4F04C0215C3F4F4F4F5F4FE1E089
:100F4000F0E0203080E0380780E0480780E4580770
:100F500028F5E0E0F0E022C0E038F1056CF5E1585A
:100F6000FF4FDA01C9018F779070A070B0708034A4
:100F70009105A105B10539F427FF09C0205C3F4F59
:100F80004F4F5F4F04C0215C3F4F4F4F5F4F57FFA4
:100F900005C05695479537952795319687E0569524
:100FA0004795379527958A95D1F70BC0E0E0F0E09B
:100FB00005C0E0E0F0E005C0EFEFF0E020E030E059
:100FC000A9018E2F879588278795942F9F776795FE
:100FD00066276795E695E22EA92FA82BFE2FF62B04
:100FE000622F732F8A2F9F2FCDB7DEB7E6E0EAC0BE
:100FF000DC01FB012C9111963C91119712968C917A
:101000001297482F4F7750E0982F991F9927991FD3
:1010100013966C911397862F880F892B90E0661F8B
:101020006627661F6183009739F521153105410553
:10103000510511F482E029C082E89FEF93838283F7
:1010400067E0220F331F441F551F6A95D1F783E0D5
:10105000808309C0220F331F441F551F8281938153
:10106000019793838283203080E0380780E048072F
:1010700080E4580778F320C08F3F910579F421155B
:1010800031054105510519F484E08083089544FF3A
:1010900003C081E0808310C010820EC08F57904043
:1010A0009383828383E0808387E0220F331F441F72
:1010B000551F8A95D1F7506424833583468357831F
:1010C0000895FC01DB019081923008F449C08C91B5
:1010D000823008F445C0943051F461818430B1F518
:1010E00011962C91119730E0261B310941C08430B4
:1010F00021F0923041F48230B1F111968C91119728
:101100008823A1F12DC06181823001F111968C916B
:1011100011976817D9F42281338112968D919C9191
:1011200013978217930794F028173907BCF024818E
:1011300035814681578114968D919D910D90BC917A
:10114000A02D82179307A407B50718F4662341F072
:101150000DC0281739074A075B0728F4662331F0CA
:1011600021E030E005C020E030E002C02FEF3FEF8B
:10117000C90108952F923F924F925F926F927F9292
:101180008F929F92AF92BF92CF92DF92EF92FF9297
:101190000F931F93CF93DF93CDB7DEB7CA1BDB0B43
:1011A0000FB6F894DEBF0FBECDBF09942A883988E8
:1011B00048885F846E847D848C849B84AA84B984EF
:1011C000C884DF80EE80FD800C811B81AA81B981FB
:1011D000CE0FD11D0FB6F894DEBF0FBECDBFED010F
:0611E0000895F894FFCF12
:0A11E60001000000000000000000FE
:00000001FF
